:100000000C9417060C941E290C944B290C943F0653
:100010000C94BF0C0C943F060C943F060C943F06C6
:100020000C943F060C943F060C943F060C943F063C
:100030000C943F060C943F060C943F060C943F062C
:100040000C9478290C943F060C94102D0C944B2D95
:100050000C943F060C943F060C943F060C943F060C
:100060000C943F060C943F06511C581C581C511C04
:10007000581C581C581C581C581C581C581C581CE0
:10008000581C581C581C581C581CC61B581C581C63
:10009000581C581C581C301B581C581C581C581CE9
:1000A000581C581C581C581C581C581C581C581CB0
:1000B000581C581C581CD21BD21BD21BD21BD21B43
:1000C000D21BD21BD21BD21B581C581C581C581CAC
:1000D000581C581C301BD11BD11BD11BD11B581CC9
:1000E000E21BEA1BF21BFA1B021C0A1C121C1A1C44
:1000F000241C2E1C381C421C751B351B581C581CFC
:10010000581C581CC61B581C581C581C581C581CE2
:10011000581C581C581CD01BD01BD01BD01B581C63
:10012000E21BEA1BF21BFA1B021C0A1C121C1A1C03
:10013000241C2E1C381C421C751B351B581C581CBB
:10014000581C581CC61B891C891C891C891C891CAD
:10015000891C891C891C891C891C891C891C891C77
:10016000A91DA91DA91DA91DA91DA91DD01CDA1C09
:10017000E41CEE1C541D5E1D6C1D7D1D1A1E8A1E86
:100180005B1E601E651E6A1E6F1E741E791E8A1E0F
:10019000841EA325B825C425CD25DA2500260826EA
:1001A0002B261826456E746572206D656E752E2E91
:1001B0002E00546F67676C6564206D6963726F50C1
:1001C000504D00546F67676C656420696E76657288
:1001D0007465642050504D2100546F67676C6564EE
:1001E000205458206D7574696E672100546F6767DD
:1001F0006C65642074656C656D657472792100505E
:10020000726F746F636F6C206572726F72207769A2
:1002100074682052580054696D656F757420776852
:10022000656E20636F6E6E656374696E6720746FB0
:1002300020525800507265737320616E79206B658F
:100240007920746F2063616E63656C00436F6E6E1E
:10025000656374696E6720746F2052582C20706F2C
:100260007765722075702074686520525820287751
:100270006974682062696E6420706C7567206966B5
:10028000206E6F74207573696E6720616C77617979
:10029000732062696E642900546F67676C6564201F
:1002A00027696D6D656469617465206F757470751B
:1002B000742700546F67676C65642027736C6176E0
:1002C00065206D6F64652700546F67676C656420F7
:1002D00027616C776179732062696E642700546FBF
:1002E00067676C65642050504D206368616E6E6571
:1002F0006C206C696D6974005365742052535349C6
:1003000020696E6A656374696F6E206368616E6EE2
:10031000656C2028303D3D64697361626C6529001D
:100320005365742050504D206D696E696D756D2058
:1003300073796E630053657420626561636F6E202C
:10034000696E74657276616C0053657420626561D4
:10035000636F6E2064656C6179005365742062651B
:1003600061636F6E206672657175656E6379206971
:100370006E20487A3A20303D64697361626C652C66
:100380002050783D504D52206368616E6E656C2040
:10039000782C2046783D465253206368616E6E6526
:1003A0006C2078005365742050574D2073746F7023
:1003B0002064656C61792028302064697361626C07
:1003C00065642C20312D323535203D3D20302E31D5
:1003D00073202D2035306D696E29005365742050CF
:1003E000504D2073746F702064656C6179202830E3
:1003F0002064697361626C65642C20312D3235355F
:10040000203D3D20302E3173202D2035306D696E1A
:100410002900536574206661696C736166652064A8
:10042000656C61792028302064697361626C656451
:100430002C20312D323535203D3D20302E3173209A
:100440002D2035306D696E29002A2A2A2A2A2A2A67
:100450002A2A2A2A2A2A2A2A2A2A2A2A2A2A2A2AFC
:100460002A2A2A2A2A2A0052582041636B656420CE
:100470002D2072657665727420737563636573737E
:1004800066756C21002A2A2A2A2A2A2A2A2A2A2A36
:100490002A2A2A2A2A2A2A2A2A2A2A2A2A2A2A2ABC
:1004A0002A2A002A2A2A2A2A2A2A2A2A2A2A2A2AD6
:1004B0002A2A2A2A2A2A2A2A2A2A2A2A2A2A2A2A9C
:1004C0000052582041636B6564202D207570646173
:1004D0007465207375636365737366756C21002A98
:1004E0002A2A2A2A2A2A2A2A2A2A2A2A2A2A2A2A6C
:1004F0002A2A2A2A2A2A2A2A2A2A2A2A0056616CE1
:1005000069642063686F69636573206172653A206E
:100510005B315D2D5B31365D20286368616E6E65F1
:100520006C20312D31362900536574206F7574703D
:10053000757420666F7220706F727420005B585D56
:100540002061626F7274206368616E6765732061F9
:100550006E64206578697420525820636F6E6669F6
:1005600067005B535D207361766520736574746901
:100570006E677320746F205258005B525D20726565
:10058000766572742052582073657474696E67734F
:1005900020746F2064656661756C747300557365B3
:1005A000206E756D62657273205B312D445D207421
:1005B0006F206564697420706F727473205B452DC1
:1005C000515D20666F722073657474696E67730085
:1005D000202D20726563656976657220636F6E6693
:1005E0006967757261746F722C207278207377203E
:1005F000000A0A6F70656E4C52536E672000536597
:10060000742073657269616C2062617564726174D3
:10061000653A200056616C69642063686F696365A0
:10062000733A2031202D20342B34202F2032202DDE
:100630002038202F2033202D20382B34202F203419
:10064000202D203132202F2035202D2031322B3407
:10065000202F2036202D203136005365742043682A
:10066000616E6E656C20636F6E6669673A20005339
:1006700065742044617461726174652028302D3284
:10068000293A200053657420486F70206368616EBA
:100690006E656C7320286D61782032342C20736570
:1006A0007061726174656420627920636F6D6D6141
:1006B00073292076616C69642076616C756573209E
:1006C000312D3235353A2000536574206368616EF0
:1006D0006E656C2073706163696E672028783130B5
:1006E0006B487A293A200053657420524620706F77
:1006F0007765722028302D37293A20005365742001
:100700005246206D616769632028686578292065F5
:100710002E672E20307844454144463030443A20FC
:10072000005365742062617365206672657175653A
:100730006E63792028696E20487A293A20005B5A36
:100740005D20656E74657220726563656976657299
:1007500020636F6E66696775726174696F6E20756C
:1007600074696C79005B465D20646973706C6179B3
:100770002061637475616C206672657175656E6366
:100780006965732075736564005B525D2063616CFD
:1007900063756C6174652072616E646F6D206B654A
:1007A0007920616E6420686F70206C697374005BDF
:1007B000495D207265696E697469616C697A65204A
:1007C00073657474696E677320746F20736B6574DE
:1007D00063682064656661756C7473005B585D20A6
:1007E000726576657274206368616E6765732061F7
:1007F0006E642065786974206D656E75005B535D6D
:1008000020736176652073657474696E67732074F4
:100810006F20454550524F4D20616E6420657869C8
:1008200074206D656E7500557365206E756D62651B
:100830007273205B302D395D20746F20656469749C
:1008400020706172616D657465727300202D205394
:10085000797374656D20636F6E6669677572617414
:10086000696F6E000A0A6F70656E4C52536E672096
:10087000005129204F7574707574206265666F721F
:1008800065206C696E6B20283D465329203A200074
:10089000502920536C617665206D6F646520286552
:1008A00078706572696D656E74616C293A20004FCD
:1008B000292054696D65642042494E4420617420AA
:1008C0007374617274757020203A20004E29205094
:1008D000504D206F7574707574206C696D69746506
:1008E0006420202020203A200044495341424C45B6
:1008F00044004D292050504D205253534920746FCD
:10090000206368616E6E656C202020203A20004CC8
:10091000292050504D206D696E696D756D20737979
:100920006E63202875732920203A200044495341E2
:10093000424C4544004B29204661696C73616665F1
:1009400020626561636F6E20696E74762E20283197
:100950002D32353573293A20004A29204661696CC9
:100960007361666520626561636F6E2064656C61AA
:10097000792028302D323535203D3E20313073200E
:100980002D203135306D696E293A200049292046E5
:1009900061696C7361666520626561636F6E206674
:1009A00072712E203A200048292050574D20737430
:1009B0006F702064656C6179202020202020203A0F
:1009C000200047292050504D2073746F70206465BB
:1009D0006C6179202020202020203A200046292008
:1009E0004661696C736166652064656C617920207D
:1009F00020202020203A200050574D206368616E4F
:100A00006E656C200066756E6374696F6E3A2000C7
:100A10002920706F72742000506F776572546F7761
:100A2000657200445446205548462033322D626991
:100A3000742031306368004F70656E4C52536E679E
:100A40005258206D696E6920342F36636800466CF9
:100A50007974726F6E2F4F72616E676552582055B0
:100A600048462038636800525820747970653A20EF
:100A70000044697361626C656400487A00203D3D02
:100A8000200043616C63756C617465642070616300
:100A90006B657420696E74657276616C3A200042F1
:100AA00029204D6963726F202868616C6629205087
:100AB000504D202020203A00412920496E76657251
:100AC0007465642050504D20696E20202020203A0B
:100AD000003029204D7574652062757A7A65722020
:100AE000286D6F73746C79293A0039292053657227
:100AF00069616C2062617564726174653A00736D3E
:100B0000617274506F7274004672536B7900547244
:100B1000616E73706172656E740044697361626CBA
:100B200065640038292054656C656D657472793A86
:100B300020202020202020003729204368616E6E6D
:100B4000656C20636F6E6669673A20200036292045
:100B500044617461726174652028302D32293A2015
:100B6000202000352920486F70206368616E6E6513
:100B70006C733A2020202020003429204368616EC5
:100B80006E656C2073706163696E673A2020003374
:100B90002920524620706F7765722028302D372922
:100BA0003A202020003229205246206D6167696377
:100BB0003A202020202020202020003129204261BE
:100BC0007365206672657175656E63793A202020C1
:100BD0000000000000240027002A0000000000257B
:100BE0000028002B0000000000230026002900043C
:100BF00004040404040404020202020202030303C4
:100C000003030301020408102040800102040810BD
:100C1000200102040810200000000700020100006B
:100C2000030406000000000000000000F32E112461
:100C30001FBECFEFD8E0DEBFCDBF13E0A0E0B1E034
:100C4000E8E2F0E602C005900D92A639B107D9F7A7
:100C500016E0A6E9B3E001C01D92A935B107E1F79E
:100C60001CE0CEE2DCE004C02297FE010E94EF2FE0
:100C7000CC32D107C9F70E94382F0C9412300C9453
:100C80000000A0E0B0E0E7E4F6E00C94BE2FEC0139
:100C9000A880B980CA80DB80A114B104C104D1044A
:100CA00041F484E2A82E89EDB82E8BE5C82E87E0AA
:100CB000D82EC601B5012DE133EF41E050E00E948E
:100CC0009B2F27EA31E440E050E00E94472F7B0150
:100CD0008C01C601B5012DE133EF41E050E00E94E7
:100CE0009B2FCA01B9012CEE34EF4FEF5FEF0E944A
:100CF000472F6E0D7F1D801F911F97FF04C061500D
:100D0000704080409048688379838A839B839B01ED
:100D1000AC015F77B901CA01CDB7DEB7EAE00C9448
:100D2000DA2F0E944106089581EB92E00E9441066D
:100D300008956093B1027093B2028093B3029093CE
:100D4000B4020895A0E0B0E0E8EAF6E00C94B72F12
:100D5000EC012B016A016115710519F0FB0191830A
:100D60008083C114D10449F0C6010297839728F00B
:100D700020E030E040E050E0DCC0A9908A2D90E017
:100D80000E940730892BC9F7FDE2AF1621F4A99024
:100D90003324339405C08BE2A81609F4A9903324B8
:100DA000C114D10421F0E0E1CE16D10411F5F0E335
:100DB000AF1669F48881883711F0883541F4A9802D
:100DC000229682E0382A20E1C22ED12C12C0C11412
:100DD000D10479F4E0E3AE1659F199E9E92E99E9E5
:100DE000F92E99E9092F99E1192F8AE0C82ED12C03
:100DF0003AC0FAE0CF16D10491F080E1C816D104D0
:100E000029F0E8E0CE16D104F9F415C0BFEFEB2EBF
:100E1000BFEFFB2EBFEF0B2FBFE01B2F24C0A9E9B4
:100E2000EA2EA9E9FA2EA9E90A2FA9E11A2F1BC077
:100E3000F8E0CF2ED12CEFEFEE2EEFEFFE2EEFEFFE
:100E40000E2FEFE11E2F0FC09601442737FD40956E
:100E5000542F6FEF7FEF8FEF9FEF0E94792FC90123
:100E6000DA017C018D0120E030E040E050E060E0FC
:100E70003601882477FC8094982C70EDB72EBA0C3C
:100E8000F9E0FB1570F48A2D81548A3118F499EC3D
:100E9000B92E06C08A2D81568A3148F589EAB82EC6
:100EA000BA0C8B2D90E08C159D050CF56F3FE9F089
:100EB000E216F30604071507B8F0CA01B901A40148
:100EC00093010E94472F9B01AC018B2D90E0A0E085
:100ED000B0E0280F391F4A1F5B1F281739074A0740
:100EE0005B0710F061E001C06FEFA990C6CF41141D
:100EF000510451F0662311F0219703C031FE04C064
:100F00002297F201D183C08330FE07C050954095EF
:100F1000309521953F4F4F4F5F4F67FF0AC082E2E8
:100F200090E090935806809357062FEF3FEF4FEFD6
:100F30005FEFB901CA01CDB7DEB7E1E10C94D32F61
:100F4000FC0188279927E89421912032E9F3293080
:100F500010F02E30C8F32B3241F02D3239F4689462
:100F600004C00E94F507820F911D219120532A3061
:100F7000C0F31EF4909581959F4F089546E953E084
:100F80000E94C3070895009731F4DA018D919C9176
:100F9000009709F40EC0DC01FB013D912191222351
:100FA00019F03217C9F3FACF332331F4DA011D9265
:100FB0001C928827992708951197AF93BF93FB013F
:100FC0003D912191321771F4332321F48827992719
:100FD000119702C01E921196FA01A193B0839F91BE
:100FE0008F910895222369F7EACF7AE0979F902D99
:100FF000879F802D910D1124089580919803813051
:1010000019F482E08093980380919803833019F457
:1010100084E0809398030895E3E0F0E089E0809312
:101020005700849190E08670863009F491E0892F12
:1010300008951F93182F0E940C08882379F09FB7FA
:1010400081E080939F05F894A89588E180936000E3
:1010500010936000112309F0A8959FBF1F91089578
:10106000382F20E080913105909132058227932717
:1010700040E061E270E19C01220F331F97FF04C042
:10108000C9018627972701C0C9014F5F483099F7EA
:101090009093320580933105089587E38093CE03C2
:1010A00080E092ECA1E0B0E08093CF039093D00376
:1010B000A093D103B093D20387E08093DB0380E059
:1010C00091EAACEBB3E38093D3039093D403A09362
:1010D000D503B093D60385E08093DC038DEE9EEFBD
:1010E000ADEABEED8093D7039093D803A093D903C4
:1010F000B093DA03ADEDB3E080E090E0863010F01D
:10110000E0E004C0FC01E058FC4FE081ED93019663
:101110008831910599F782E08093F5038AE0809306
:10112000F603089580E09EECADEEB4E380939B035C
:1011300090939C03A0939D03B0939E0380E090E066
:10114000A0E0B0E580939F039093A003A093A10338
:10115000B093A203E3EAF3E080E081938F5F8031F4
:10116000E1F708958436910520F4BC0180E090E019
:1011700025C08E3B910550F48A559040BC0180E01B
:1011800090E02AE030E040E050E016C0823D91055A
:1011900050F4845B9040BC0180E090E024E630E0B5
:1011A00040E050E009C08D5C9040BC0180E090E0E0
:1011B00028E532E040E050E00E94472F24E630E08E
:1011C00040E050E00E94472F089590E08C599F4FD7
:1011D0000E94B2080895DC019896EC91F0E0E77067
:1011E000F070E858FC4F808108958F929F92AF92E3
:1011F000BF92CF92DF92EF92FF920F931F938C01D9
:101200000E94EB08D80197962C9130E043E150E022
:10121000249FF001259FF00D349FF00D1124EB5415
:10122000FD4F80809180A280B38090E00F96AA2726
:1012300097FDA095BA2FBC01CD0120E43FE14DE719
:1012400050E00E94472FA50194010E94792F690167
:101250007A0180ED97E0A0E0B0E0C80ED91EEA1E4A
:10126000FB1ED80198968C91887181F060E07EEE2B
:101270008AEB9BE0A50194010E94792F28513C4FF5
:101280004F4F5F4FC20ED31EE41EF51E87EE93E054
:10129000A0E0B0E0C80ED91EEA1EFB1EC701B601D1
:1012A00028EE33E040E050E00E94792FCA01B901F6
:1012B00028EE33E040E050E00E94472F1F910F914D
:1012C000FF90EF90DF90CF90BF90AF909F908F9066
:1012D00008958F3F910509F010F480E0089522E011
:1012E0008030920710F481E008958050934010F010
:1012F00083E0089582E00895CF92DF92FF920F93EA
:101300001F93CF93DF93F82FEB016A01182F1695E7
:10131000E0E088819981D6018C938A819B81119626
:101320008C9311978C819D8112968C9312978E814C
:101330009F8113968C931397288139814A815B8111
:101340006C817D818E819F819295990F990F907C00
:10135000832F8370982B852F8370880F880F982B8D
:10136000872F83708295807F982B14969C9385E0BD
:1013700090E0C80ED91E2896EF5F1E1750F6F0FFBA
:1013800021C0888199810E946909F82E8A819B81F8
:101390000E946909182F8C819D810E946909082F7C
:1013A0008E819F810E946909F294FF0CFF0C70EC02
:1013B000F7221295107F1F29182B000F000F012B09
:1013C000D6010C93DF91CF911F910F91FF90DF9089
:1013D000CF90089523E08032920718F420E030E0A7
:1013E00026C023E0883E920748F49C012F513340E9
:1013F00054E0369527955A95E1F719C027E0803DCE
:10140000920720F49C012C5D334011C028E08839FC
:10141000920718F02FEF33E00AC09C01285C374098
:1014200044E0369527954A95E1F72D503C4FC90188
:1014300008958C30910548F49C0174E0220F331F0D
:101440007A95E1F7285D3C4F17C023E0843F92076F
:1014500020F49C0124523C4F0FC024E080309207BE
:1014600018F020E938E008C09C012657334F64E0AB
:10147000220F331F6A95E1F7C90108959C01369543
:10148000279525753575821B930B9C0136952795FD
:10149000369527952373337383739373280F391FFE
:1014A000C901E4E096958795EA95E1F7820F931FCD
:1014B0008F709F7021E031E0AC01429FC001439FDB
:1014C000900D529F900D1124892F0895882339F093
:1014D0005A980000419A00005A9A000008955A98BC
:1014E0000000419800005A9A000008955A9A00009E
:1014F00086B15A980000817008950F931F93082FAA
:101500005C9A5A985C9810E0802F80780E94660A56
:10151000000F1F5F1830C1F75A981F910F9108955F
:101520008F770E947D0A08950F931F93082F10E074
:10153000802F80780E94660A000F1F5F1830C1F765
:101540005A981F910F9108950F931F935A9880E016
:1015500000E0182F110F0E94760A810F0F5F0830EC
:10156000C1F71F910F9108950E94900A0E94A40A4A
:101570005C9A08951F93162F80680E947D0A812F20
:101580000E94940A5C9A1F9108951F931091D703AB
:101590001827EEECF3E0E80FF11D89E767850E945C
:1015A000BA0A8DE3612F0E94BA0A82E4612F0E9479
:1015B000BA0A1F91089586E20E94B40A08950F9313
:1015C0001F938C018CE1F80164810E94BA0A8DE1BD
:1015D000F80165810E94BA0A8EE1F80166810E94D5
:1015E000BA0A80E2F80167810E94BA0A81E2F80132
:1015F00060850E94BA0A82E2F80161850E94BA0AF7
:1016000083E2F80162850E94BA0A84E2F8016385E8
:101610000E94BA0A85E2F80164850E94BA0A8AE249
:10162000F80165850E94BA0A8EE6F80166850E9477
:10163000BA0A8FE6F80167850E94BA0A80E7F801C6
:1016400060890E94BA0A81E7F80161890E94BA0A9A
:1016500082E7F80162890E94BA0A1F910F910895EA
:10166000EF92FF920F931F93CF93DF937B018C0137
:10167000603028E372072CE982072CE1920728F5F5
:1016800020E836E948E950E00E94792FE90168979F
:10169000B90180E090E020E839E647E65FEF0E947C
:1016A000472F6E0D7F1D801F911F22E0660F771F51
:1016B000881F991F2A95D1F721E732E040E050E0DA
:1016C0000E94792F890180E421C020E03DE241E3BE
:1016D00051E00E94792FE9016897B90180E090E01C
:1016E00020E033ED4EEC5EEF0E94472F6E0D7F1D24
:1016F000801F911F660F771F881F991F21E732E017
:1017000040E050E00E94792F890180E69E012F7110
:10171000622F680F85E70E94BA0A86E7612F0E9450
:10172000BA0A87E7602F0E94BA0ACDB7DEB7E6E0B3
:101730000C94DE2F682F8DE60E94BA0A08959F92BE
:10174000AF92BF92CF92DF920F93DF93CF9300D0EF
:1017500000D0CDB7DEB7982E83E00E94B40A809304
:10176000F70384E00E94B40A8093F80386E060E007
:101770000E94BA0A87E061E00E94BA0A89E06FE736
:101780000E94BA0A8AE065E00E94BA0A8BE062E130
:101790000E94BA0A8CE065E10E94BA0A8DE06DEF02
:1017A0000E94BA0A8EE060E00E94BA0A992019F0FD
:1017B00084E193E008C08091F50323E1829FC0019A
:1017C00011248B549D4F0E94DF0A80E36CE80E9435
:1017D000BA0A82E36FE00E94BA0A83E362E40E94DD
:1017E000BA0A84E36AE00E94BA0A85E36AE20E94C8
:1017F000BA0A86E36DE20E94BA0A87E364ED0E94AA
:10180000BA0A88E360E00E94BA0A89E360E00E94B5
:10181000BA0A992049F055E8A52E51ECB52E51ECA5
:10182000C52E5EEDD52E08C0A090D703B090D8038A
:10183000C090D903D090DA030AE38D2D9927AA2707
:10184000BB2789839A83AB83BC83802F69810E94E5
:10185000BA0A802F8B5F69810E94BA0ADC2CCB2CDC
:10186000BA2CAA240F5F0E3341F783E46FEF0E9476
:10187000BA0A84E46FEF0E94BA0A85E46FEF0E940F
:10188000BA0A86E46FEF0E94BA0A992019F08DE631
:1018900066E003C08DE66091DB030E94BA0A89E727
:1018A00060E00E94BA0A8AE76091DC030E94BA0AEB
:1018B00083E760E00E94BA0A84E760E00E94BA0A07
:1018C000992029F060E071EA8CEB93E308C0609105
:1018D000D3037091D4038091D5039091D6030E94D5
:1018E000300B0F900F900F900F90CF91DF910F91D1
:1018F000DF90CF90BF90AF909F90089587E061E018
:101900000E94BA0A8EE764E20E94BA0A88E063E0A5
:101910000E94BA0A88E060E00E94BA0A87E065E0A7
:101920000E94BA0A85E062E00E94BA0A83E00E943F
:10193000B40A8093F70384E00E94B40A8093F8030A
:101940000895582F40919C04842F90E0FC01EF7083
:10195000F0709F012F5F3F4F64E0959587956A95E2
:10196000E1F72817390751F0E457FB4F5083842FD4
:101970008F5F8F70407F842B80939C0408951F920B
:101980000F920FB60F921124EF92FF920F931F93B5
:101990002F933F934F935F936F937F938F939F9377
:1019A000AF93BF93EF93FF93E0909F03F090A0035A
:1019B0000091A1031091A20386B1A80197012074A0
:1019C00030704070507090E065E0969587956A950C
:1019D000E1F7A0E0B0E081709070A070B0702817BF
:1019E00039074A075B0709F46AC0209184003091E7
:1019F000850010928500109284008091BF04882396
:101A000009F05DC0E5FC02C03695279589E0253CCC
:101A10003807C8F180914703A8019701BCE15695AA
:101A2000479537952795BA95D1F721153105410589
:101A3000510521F421E030E040E050E090E0A0E0EA
:101A4000B0E0281739074A075B07D0F480914703B5
:101A50008F3FB1F020E00EC0E22FF0E0EE0FFF1F4D
:101A6000DF01A054BB4F8D919C91E95DFC4F9183A8
:101A700080832F5F80914703281770F31092BE0474
:101A8000109247031CC082E02D3B3807A8F08091DC
:101A90004703803188F410914703C9010E94EA0985
:101AA000E12FF0E0EE0FFF1FE054FB4F91838083A6
:101AB0001F5F1093470303C08FEF80934703FF918D
:101AC000EF91BF91AF919F918F917F916F915F91B6
:101AD0004F913F912F911F910F91FF90EF900F9099
:101AE0000FBE0F901F90189583E0809380008AE1CD
:101AF000809381008FEF9FEF9093890080938800FF
:101B000010926F0080E280936C00E8E6F0E0808144
:101B10008260808308956F3018F08695805808950C
:101B200089E0689F802D11240895E82FF0E0E656A3
:101B3000FC4FE185E03118F0E0E0F2E00AC0F894F3
:101B4000F0E0EE0FFF1FE95DFC4F0190F081E02D0A
:101B50007894CF010895882319F460E071E002C001
:101B600063E071E085E396E00E94FB2C0895A0E01D
:101B7000B0E0EDEBFDE00C94C02F182F0E94CE29B1
:101B80009B01AC0180912B0590912C05A0912D0516
:101B9000B0912E0569017A01C81AD90AEA0AFB0A2E
:101BA000D701C60189589341A040B04010F010926F
:101BB0002A0520932B0530932C0540932D05509337
:101BC0002E052091BF04822F81508230E8F580914C
:101BD0002A05882309F44FC1813011F482E0BCC189
:101BE000803108F035C1E82FF0E0E054FB4F10835E
:101BF0008F5F80932A05803109F0B0C1A2ECB4E078
:101C0000213039F41196EC911197E695E6958C9177
:101C100009C08D919C911197E92FE695E695E6957F
:101C200096958795E03140F4F0E090E0EE0FFF1FCD
:101C3000E95DFC4F918380831092BE04129684E08C
:101C4000A03DB807E9F68AC1233009F004C18091AC
:101C50002A05882321F41F3009F080C10CC1883186
:101C600030F4E82FF0E0E154FB4F108374C1883169
:101C700009F0EEC0112309F0EBC0C0E0D0E00BE0AA
:101C800010E0DE0163E0AA0FBB1F6A95E1F7C09F79
:101C9000B001C19F700DD09F700D1124FB01E05465
:101CA000FB4F80812181922F977095958795FD013B
:101CB000EE0FFF1FE95DFC4F91838083FB01EF5323
:101CC000FB4F30813695369536952181422F4295CE
:101CD000440F407E842F832B269526952695922FA0
:101CE000977095958795FD01EE0FFF1FE75DFC4FFF
:101CF00091838083FB01EE53FB4F80818295869513
:101D0000869583704181942F990F990F292F282B45
:101D1000429546954695437082818170880F880F61
:101D2000382F342B35952795FD01EE0FFF1FE55D0C
:101D3000FC4F31832083FB01EC53FB4F3081369500
:101D40002181422F479544274795842F832B269541
:101D5000922F977095958795FD01EE0FFF1FE35D1C
:101D6000FC4F91838083FB01EB53FB4F3081329515
:101D70003F702181422F4295407F842F832B2295F3
:101D80002F70922F977095958795FD01EE0FFF1F8D
:101D9000E15DFC4F91838083FB01EA53FB4F80811F
:101DA000881F8827881F4181942F990F292F282B5E
:101DB000441F4427441F82818370880F382F342B9F
:101DC00035952795FD01EE0FFF1FEF5CFC4F31832A
:101DD0002083FB01E853FB4F3081369536952181F6
:101DE000422F4295440F440F407C842F832B26952D
:101DF0002695922F977095958795AA0FBB1FFD0189
:101E0000ED5CFC4F9183808367537B4FFB01208106
:101E10002295269527704181342F330F330F330FCE
:101E2000832F822B942F92959695977095958795F1
:101E3000AB5CBC4F11969C938E932196C230D1051A
:101E400009F01FCF8091D60483FD02C01092BE041A
:101E500010922A0583C0243009F080C040912A05E1
:101E6000442359F4183AB1F4109232051092310516
:101E700088EA0E94300881E06FC0413019F4109365
:101E80002F0504C0423031F410933005812F0E9499
:101E900030085DC060913005262F30E0220F331FDF
:101EA000E42FF0E0C90102968E179F0734F0433209
:101EB00068F7E354FB4F1083E9CF2D5F3F4F40910C
:101EC000310550913205E217F30749F4912F80E074
:101ED00048275927509332054093310538C0812F48
:101EE00090E04817590789F580912F05813069F5F1
:101EF000613118F080E180933005D090300510EC0E
:101F0000E12E14E0F12E00E010E01BC0F701D081BB
:101F1000C0E0818190E08C2B9D2BB3E09695879556
:101F2000BA95E1F70E94EA09F801EE0FFF1FE95D9B
:101F3000FC4F918380830F5F1F4F82E090E0E80E9B
:101F4000F91E0D1518F31092BE0410922A05809107
:101F50002A05882319F08F5F80932A05CDB7DEB755
:101F6000E8E00C94DC2FFF920F931F93CF93DF9345
:101F7000182F092FF62E8EE30E94BA0A212F302F38
:101F8000C901EC0110E005C08FE769910E94BA0A0F
:101F90001F5F1F15C8F385E064E00E94BA0A83E062
:101FA0000E94B40A8093F70384E00E94B40A8093ED
:101FB000F8030E94CE296093F9037093FA0380938B
:101FC000FB039093FC0387E069E00E94BA0A81E07A
:101FD00080939803CDB7DEB7E5E00C94DF2F0E9425
:101FE000B30F809198038130D9F40E94CE292091BB
:101FF000F9033091FA034091FB035091FC03621BFB
:10200000730B840B950B605A76488140904040F4E6
:10201000E8CF85E396E067E071E00E94FB2C08952D
:10202000809198038130A9F3089585E396E06EE7E7
:102030000E94B32E0895A0E0B0E0E1E2F0E10C943C
:10204000BF2F6C0185E396E06EE70E94B32E760108
:1020500000E010E0C0E0D0E0B0E2BB2E0AC00830E3
:10206000110521F49E012095F60120870894E11CBA
:10207000F11CF7016081862F8D57823040F485E393
:1020800096E06DE70E94B32EF70160816B2585E332
:1020900096E00E94B32E0115110551F0F7018081E1
:1020A0009E01280F311DC32FDD27C20FD31FD07013
:1020B0000F5F1F4F0930110591F6CDB7DEB7E9E08C
:1020C0000C94DB2FA9E0B0E0E8E6F0E10C94C62F19
:1020D000382FE62F8091A10490E0019664E270E031
:1020E0000E94662F982F8093A10488E9898380E15C
:1020F0008A83913071F0913028F0923099F09330CA
:10210000E1F416C085E08B8381EF8C832F5F2D83F4
:1021100017C09B8381EF8C8384E6489FC001112404
:102120009D830EC084E08B8381EF8C833D8308C048
:102130009B8381EF8C83ED8303C00E94151004C044
:10214000CE0101960E941B102996E2E00C94E22F2A
:102150000F931F93CF93DF93182F092F85E396E0FA
:102160006EE70E94B32E212F302FC901EC0110E041
:1021700000E288818D57823040F485E396E06DE778
:102180000E94B32E88818027888385E396E0699139
:102190000E94B32E1F5F193061F785E396E06EE76A
:1021A0000E94B32EDF91CF911F910F910895A9E066
:1021B000B0E0EDEDF0E10C94C62F382F8091A10432
:1021C000882379F48EEF89833A836B83842F90E0A0
:1021D000959587958C832D83198618861F821E827C
:1021E0002FC040919C04842F90E09C012F70307090
:1021F00054E0959587955A95E1F78217930721F159
:102200008DEF89831A821B82DE01149620E008C0BC
:10221000E457FB4F80818D93405F2F5F263069F03C
:10222000842F90E0FC0134E0F595E7953A95E1F7CD
:102230008F709070E817F90759F740939C042A8330
:10224000CE0101960E94A8108091A10490E0019611
:1022500066E070E00E94662F8093A1042996E2E078
:102260000C94E22F9F92AF92BF92CF92DF92EF92A7
:10227000FF920F931F93B82EA62ED42EC22E902E0F
:102280000E94CE297B018C0180918B0420919D04BA
:1022900030919E0440919F045091A0048823B1F096
:1022A000D801C701821B930BA40BB50B815E9E4224
:1022B000A040B04020F12C2DDC1408F42D2D8B2DE6
:1022C0006A2D422F292D0E94621011C0D801C7012A
:1022D000821B930BA40BB50B81539547A040B040D4
:1022E00070F08B2D6A2D4D2D2C2D0E94D710E09271
:1022F0009D04F0929E0400939F041093A0041F91EC
:102300000F91FF90EF90DF90CF90BF90AF909F9094
:10231000089585E396E06091FE030E94B32E089530
:102320001F93182F85E396E0612F0E94B32E8091B2
:10233000FE0381278093FE031F9108951F93192F99
:102340000E949011812F0E9490111F910895DF9299
:10235000EF92FF920F931F93D82E7B011092FE03F2
:1023600005E316E0C80165EB0E94B32EC80162E6E2
:102370000E94B32E8D2D0E949011C7010E949E11C4
:102380001F910F91FF90EF90DF9008958EE060E035
:102390000E94532A8FE061E00E94532A82E061E0AC
:1023A0000E94532A83E060E00E94532A84E061E0A7
:1023B0000E94532A0895892B19F089E061E002C038
:1023C00089E060E00E94BF2A0895A0E2B0E0EBEE51
:1023D000F1E10C94BE2F8CE00E94B40A882379F5B9
:1023E00085E396E063E171E00E94FB2C2C9A80E08B
:1023F0000E949F0B0E947E0C2C9821C085E396E0E2
:102400000E947A2E482F8091BF04882321F0842FC8
:102410000E94B70D14C080912805E82FF0E0319696
:102420009F012F71307031978091270590E0281718
:10243000390729F0E250FB4F40832093280585E3BC
:1024400096E00E94402E892BC9F680919803843033
:1024500009F08EC00E94CE296093AE047093AF0441
:102460008093B0049093B1046115710581059105C5
:1024700061F481E090E0A0E0B0E08093AE0490933E
:10248000AF04A093B004B093B1048091BA049091CA
:10249000BB0481609093BB048093BA0483E0809373
:1024A00098038FE70E94900A05EF14E00E94A40AA7
:1024B000F80181938F01F4E00E3F1F07B9F74091B7
:1024C000E0048091F504282F30E0842F90E08227EB
:1024D000932786FF40C080E448274093E004C90169
:1024E00088739070C89709F510E014C01F5F809141
:1024F000F603E12FF0E084FF06C0EB50FB4F808134
:102500000E94A10C07C0EB50FB4F85E396E0608171
:102510000E94B32E212F30E08091F50490E0877067
:1025200090708217930714F716C02F733070232B07
:1025300091F48091F6048093B2048091F704809323
:10254000B4048091F8048093B5048091FB048093D7
:10255000BC041092BD0480912905813019F482E0F9
:102560008093290580912905833011F41092290563
:102570000E94CE295B016C018091B6049091B70452
:10258000A091B804B091B9040097A105B105C9F0B4
:1025900086017501E81AF90A0A0B1B0BD801C7015D
:1025A000885B9B40A040B04060F00E94DB0A8093B3
:1025B000B3041092B6041092B7041092B8041092AB
:1025C000B9048EEC93E00E94F5082091AA043091A2
:1025D000AB044091AC045091AD0486017501E21A40
:1025E000F30A040B150BE616F7060807190708F49B
:1025F00024C1A092AA04B092AB04C092AC04D092C1
:10260000AD04A8958091BE048830A0F080919F030E
:102610009091A003A091A103B091A203ECE1B69523
:10262000A79597958795EA95D1F70097A105B105EC
:1026300009F0A2C18091BE048F5F8093BE04E09038
:10264000AE04F090AF040091B0041091B104E11415
:10265000F1040105110511F18EEC93E00E94F508DB
:10266000AE18BF08C00AD10A6A157B058C059D0506
:1026700088F480919F0384FD04C080ED97E00E9460
:10268000DB111092AE041092AF041092B0041092BD
:10269000B10404C080E090E00E94DB119091E0045E
:1026A000907C9093E0040091280510912705011774
:1026B000B1F180912905823091F590589093E00412
:1026C0008EEC93E00E94EB08893010F048E002C0E5
:1026D000482F415030E013C03F5FA32FB0E0812F5F
:1026E00090E0FC01E250FB4F2081FD01E052FB4FE6
:1026F0002083A25EBA4F2C930196182F1F713417B6
:1027000010F4101749F710932705832F895C9091D7
:10271000E004892B8093E00430931E051AC02091B9
:1027200029052430D1F490911E05EFE1F5E0A1EEEA
:10273000B4E0292F30E02E0F3F1F02C081918D930E
:10274000E217F307D9F7995C8091E004982B9093F6
:10275000E00483E08093290536C08091A50482308F
:1027600059F491609093E0042C9A03EA13E07E01FF
:102770000894E11CF11C10C09093E0042C982223D3
:1027800019F481E08093290580912905833069F748
:1027900084E080932905E9CFF80181918F010E949F
:1027A000950DF701819391937F01F3E0033B1F07A0
:1027B00099F78091F6038770BE016F5F7F4F41EEFE
:1027C00054E00E947C092B9A2091A3042223A1F0BB
:1027D0009091DB03992381F08091A4048F5F809313
:1027E000A4048150821729F41092A404892F8150E7
:1027F00001C0892F0E949A0B8091A2040E94C50AF1
:102800008EEC93E00E94EB08682F80EE94E00E942B
:10281000B30FE091A204EF5FE093A204E83131F03E
:10282000F0E0E253FC4F8785882339F41092A2042C
:1028300004C02C9A89E08093BE048091F6038871CD
:1028400071F180919803823051F58091BA04909192
:10285000BB04880F991F9093BB048093BA0483E054
:10286000809398030E947E0C0E94CE296093B60448
:102870007093B7048093B8049093B90461157105FF
:102880008105910561F481E090E0A0E0B0E08093E3
:10289000B6049093B704A093B804B093B9048091A0
:1028A000F60384FF1EC08091BA049091BB048E7F12
:1028B0000E943E0A182F8091B2046091BC040E94CD
:1028C0008B0D082F8091B304612F0E948B0D282F50
:1028D0008091B4046091B504402F009199030E9447
:1028E00032112B988091A5048130D1F0813020F0F5
:1028F000823009F047C034C08AE00E94F22A892B56
:1029000009F040C081E08093A5040E94C029609333
:10291000A6047093A7048093A8049093A90432C0DE
:102920008AE00E94F22A892B21F50E94C029209179
:10293000A6043091A7044091A8045091A904621BF9
:10294000730B840B950B695E734080409040D0F010
:1029500082E08093A50480ED97E00E94DB1112C015
:102960008AE00E94F22A892B69F080E090E00E94C0
:10297000DB111092A50406C08091BE04883009F0D6
:1029800059CF57CFA096EAE00C94DA2F89E061E0A6
:102990000E94532A89E060E00E94BF2A08951F9395
:1029A000182F0E94CE2960939D0470939E048093FB
:1029B0009F049093A00410938B04112329F440E802
:1029C00055E260E070E004C040E051EE60E070E08D
:1029D00085E396E00E94B92D1F910895ACE1B0E027
:1029E000E4EFF4E10C94BE2F0E94CE297B018C0110
:1029F00081E00E949F0BB4E7AB2E6E010894C11CCE
:102A0000D11CA3E0BA2EA982C60161E00E94EF0F9B
:102A1000B09298030E947E0C6AEF70E080E090E034
:102A20000E94F42980919803833009F07DC085E3EA
:102A300096E00E94402E892B09F076C00E94CE2994
:102A40006E197F09800B910B6058734C894C914033
:102A500008F06AC0D8CF8FE70E94900A0E94A40AAB
:102A6000843509F05CC089830E94A40A182F00E015
:102A700010932204009321040E94A40A080F111D40
:102A800010932204009321040E94A40A809320043E
:102A90000E94A40A80931F04813108F040C0FF24E3
:102AA00007C00E94A40A01501C4FF8018083F394D0
:102AB0000F2D10E080911F0490E0880F991F0817D8
:102AC000190778F380E78983CE01019661E00E94BF
:102AD000EF0F83E0809398030E947E0C62E370E026
:102AE00080E090E00E94F429809198038330A9F05F
:102AF0008FE70E94900A0E94A40A803581F489839E
:102B000003EB13E00E94A40AF80181938F01F3E024
:102B10000E3C1F07B9F781E003C082E001C083E0EB
:102B20006C96EAE00C94DA2F80919803833009F0D8
:102B300092CFF3CF83E00E94B40A8093F70384E03E
:102B40000E94B40A8093F80387E061E00E94BA0A09
:102B50006AE070E080E090E00E94F4290E947E0C20
:102B6000000008950F931F93082F17C02C9A64E656
:102B700070E080E090E00E94F4292C9864E670E018
:102B800080E090E00E94F4291F5F101778F36CE258
:102B900071E080E090E00E94F42910E0F6CF482F29
:102BA000392F25E00DC0F999FECF1FBA842F932F3E
:102BB00092BD81BD60BD0FB6F894FA9AF99A0FBE26
:102BC000215059F0F999FECF842F932F92BD81BDEA
:102BD000F89A80B5681739F7089582E00E94B21517
:102BE0000895A0E0B0E0E7EFF5E10C94B72F482E90
:102BF000562ECC24DD24EE24FF2488249924C0E022
:102C0000D0E046E4342E04C0CC24DD245524539473
:102C1000442069F480919903839DE00111243AE9ED
:102C2000E32E33E0F32E29E1822E912C1DC021E00A
:102C3000421671F480919903839DE00111246B96F3
:102C40009EECE92E93E0F92E89E2882E912C0CC09F
:102C500032E0431649F409E9E02E03E0F02E11E0DA
:102C6000812E912CC8E1D1E03E016C0C7D1C1092AC
:102C7000320510923105E3011BC0552059F4F99932
:102C8000FECFD2BDC1BDF89A80B5F701E00FF11FAC
:102C9000808307C0F701E00FF11FCE0160810E9421
:102CA000CF150E0D1F1DF80180810E94300821965E
:102CB0009E012619022F10E008151905F0F2CE0129
:102CC0005520D9F4F999FECFD2BDC1BDF89A20B5EF
:102CD000F999FECF2196D2BDC1BD2197F89A80B552
:102CE00090E0B22EAA248A299B29209131053091A7
:102CF00032052817390759F487CF2196609132059C
:102D00000E94CF15CE01609131050E94CF1580E25F
:102D100091E0C80ED91E91EEC91692E0D90608F4CA
:102D200077CF852DCDB7DEB7E1E10C94D32F80E0CE
:102D300061E00E94F11581E061E00E94F1150895C3
:102D400082E061E00E94F115089582E060E00E9457
:102D5000F11580919903843020F0109299030E941C
:102D6000A01608951F93182F0E94A516809199030D
:102D7000811731F0143020F4109399030E94A016AB
:102D80001F9108951092890485E6E4E2F4E0DF01E2
:102D90001D928A95E9F708951F93182F8F3711F028
:102DA0008830E1F5E0918904EE2309F455C0E15043
:102DB000E0938904F0E0EC5DFB4F108285E396E040
:102DC0006DE00E94B32E10E00AC0E12FF0E0EC5D50
:102DD000FB4F85E396E060810E94B32E1F5F8091D8
:102DE0008904181790F385E396E060E20E94B32E01
:102DF00085E396E06DE00E94B32E10E00AC0E12F5B
:102E0000F0E0EC5DFB4F85E396E060810E94B32E1D
:102E10001F5F80918904181790F31CC08B3119F43F
:102E20000E94C2161FC08D30E9F08A30D9F080911F
:102E30008904843688F485E396E0612F0E94B32EDE
:102E400080918904E82FF0E0EC5DFB4F10838F5FE9
:102E50008093890480E007C085E396E067E00E94E4
:102E6000672BF8CF81E01F9108951F93CF93DF93D5
:102E7000CDEDD3E010E03BC085E396E062E271E087
:102E80000E94F82C85E396E0612F4AE050E00E9412
:102E9000752C85E396E06FE271E00E94F82C699151
:102EA00070E080E090E02091DC0330E040E050E012
:102EB0000E94472F20E137E240E050E00E94472F78
:102EC000DC01CB014091D3035091D4036091D50331
:102ED0007091D603480F591F6A1F7B1F85E396E048
:102EE0002AE030E00E943C2C1F5F183119F08881E5
:102EF000882311F6DF91CF911F910895EF92FF92F1
:102F00000F931F93882339F485E396E061E77AE015
:102F10000E94852B3BC090E00E94B20824E630E07E
:102F200040E050E00E94792F122F032FF42EE52E5F
:102F3000622F732F842F952F2AE030E040E050E07D
:102F40000E94792F85E396E0BA01A9012AE030E0DA
:102F50000E942D2C85E396E06EE20E94672B612F84
:102F6000702F8F2D9E2D2AE030E040E050E00E942F
:102F7000792FAB01BC0185E396E02AE030E00E94A6
:102F80002D2C85E396E063E70E94992B1F910F910A
:102F9000FF90EF900895FF920F931F93CF93DF93CD
:102FA00085E396E067E67AE00E94462B8091B303C2
:102FB000813041F485E396E06EE47AE00E94852B4F
:102FC000FF246DC0823029F485E396E067E37AE060
:102FD000F5CF843029F485E396E063E27AE0EECF22
:102FE000853071F785E396E068E17AE0E7CFCF2D91
:102FF000D0E0C930D1051CF06F2D685C02C06F2D88
:103000006F5C85E396E00E94672B85E396E060E1C4
:103010007AE00E94462BBE016F5F7F4F85E396E00A
:103020004AE050E00E94D12C85E396E065E07AE02A
:103030000E94462B8E010D541C4FD8011196EC9125
:10304000E032F8F485E396E068EF79E00E94462BE1
:10305000F8018181803130F085E396E063E371E02F
:103060000E94F82CCD54DC4F698170E06F70707055
:103070006F5F7F4F85E396E04AE050E00E94E42CCA
:103080000DC0F0E0EF70F070EE0FFF1FE85BFC4F3B
:103090006081718185E396E00E94FB2CF39480911E
:1030A0002004F81608F4A3CF85E396E06DED79E0EF
:1030B0000E94462B8091CB030E947E1785E396E009
:1030C00062EC79E00E94462B8091CC030E947E172F
:1030D00085E396E067EA79E00E94462B8091CD0374
:1030E0000E947E1785E396E06CE879E00E94462B0B
:1030F0004091C3035091C4036091C5037091C6030E
:10310000411551056105710539F185E396E02AE025
:1031100030E00E943C2C85E396E069E579E00E946E
:10312000462B8091C7030E94E508AB01BC0185E3F3
:1031300096E02AE030E00E943C2C85E396E065E3CF
:1031400079E00E94462B85E396E06091C8034AE04F
:1031500050E00E94872C06C085E396E06CE279E09F
:103160000E94852B85E396E06FE079E00E94462B74
:103170006091C9037091CA0385E396E04AE050E08C
:103180000E94612C85E396E062EF78E00E94462B76
:103190006091C203603450F470E06F5F7F4F85E34D
:1031A00096E04AE050E00E94E42C06C085E396E0F9
:1031B00069EE78E00E94852B85E396E06CEC78E080
:1031C0000E94462B8091C10380FD03C065E371E03E
:1031D00002C069E371E085E396E00E94FB2C85E381
:1031E00096E06FEA78E00E94462B8091C1038270DE
:1031F0000E94AB0D85E396E060E978E00E94462BE3
:103200008091C10384700E94AB0D85E396E061E775
:1032100078E00E94462B8091C10388700E94AB0D1C
:10322000CDB7DEB7E5E00C94DF2F1F93CF93DF938C
:1032300085E396E06BEB7BE00E94462B4091D30345
:103240005091D4036091D5037091D60385E396E045
:103250002AE030E00E943C2C85E396E065EA7BE0C2
:103260000E94462B4091D7035091D8036091D90317
:103270007091DA0385E396E020E130E00E943C2C77
:1032800085E396E06FE87BE00E94462B85E396E0BD
:103290006091DB034AE050E00E94872C85E396E0D2
:1032A00069E77BE00E94462B85E396E06091DC03B2
:1032B0004AE050E00E94872C85E396E063E67BE0DD
:1032C0000E94462BCDEDD3E010E012C0112331F067
:1032D00085E396E06DE371E00E94F82C85E396E0CB
:1032E00069914AE050E00E94752C1F5F183119F077
:1032F0008881882359F785E396E00E946F2B85E348
:1033000096E06DE47BE00E94462B85E396E06091B9
:10331000F5034AE050E00E94872C85E396E068E3DD
:103320007BE00E94462BE091F603F0E0E770F0703E
:10333000EE0FFF1FE859FC4F6081718185E396E035
:103340000E94FB2C85E396E063E27BE00E94462B23
:103350008091F60390E0887190708830910589F033
:10336000893091051CF4892B39F01BC080319105FF
:1033700069F04897B1F40FC085E396E06AE17BE01D
:103380000EC085E396E06EE07BE009C085E396E041
:1033900068E07BE004C085E396E06EEF7AE00E948F
:1033A000852B85E396E06AEE7AE00E94462B4091F9
:1033B000CF035091D0036091D1037091D20385E384
:1033C00096E02AE030E00E943C2C85E396E061ED37
:1033D0007AE00E94462B80919F0380710E94AB0D82
:1033E00085E396E068EB7AE00E94462B80919F038C
:1033F00080740E94AB0D85E396E06FE97AE00E944D
:10340000462B80919F0380720E94AB0D85E396E06E
:1034100062E87AE00E94462B8EEC93E00E94F50869
:10342000AB01BC0185E396E02AE030E00E942D2C40
:1034300085E396E06DE77AE00E94462B8EEC93E000
:103440000E94F5089B01AC0160E472E48FE090E01B
:103450000E94792F85E396E0BA01A9012AE030E0C5
:103460000E942D2C85E396E06AE77AE00E94852B86
:10347000DF91CF911F910895EF92FF920F931F93C9
:103480007C0105E316E0C8016F2D70E04AE050E0D2
:103490000E94502CC8016EE20E94672BB701E4E045
:1034A00076956795EA95E1F76F707070C8014AE00C
:1034B00050E00E94502CC8016EE20E94672B8FE002
:1034C000E822FF24C801B7014AE050E00E94502CD6
:1034D0001F910F91FF90EF9008950F931F93CF933B
:1034E000DF93209123042F3FA9F585E396E061EF58
:1034F00075E00E94462B83E793E00E943C1A85E327
:1035000096E060ED75E00E94462B80912104909139
:1035100022040E943C1A85E396E06DE975E00E9462
:10352000852B85E396E06AE775E00E94852B85E3AD
:1035300096E062E675E00E94852B85E396E06DE3F8
:1035400075E00E94852B85E396E00E946F2B0E9418
:10355000CB1769C012160CF066C0332727FD3095D3
:103560008091200490E0821793070CF45CC085E3FF
:1035700096E068E275E00E94462B6091230477276D
:1035800067FD709585E396E04AE050E00E94E42CE8
:1035900085E396E06DEF74E00E94462B08E210E0B0
:1035A0003AC0C12FD0E0CC0FDD1FC150DC4F2881C5
:1035B00030E080912304992787FD90950197281783
:1035C000390741F585E396E06FE371E00E94F82C3E
:1035D00085E396E0602F4AE050E00E94752C85E379
:1035E00096E063E471E00E94F82CE981F0E0EF706E
:1035F000F070EE0FFF1FE85BFC4F6081718185E387
:1036000096E00E94F82C85E396E067E471E00E9462
:10361000F82C0F5F1F5F80911F04181710F285E3CD
:1036200096E00E946F2BDF91CF911F910F9108952B
:10363000ACE1B0E0EEE1FBE10C94C02F282F8091CB
:1036400023048F3F09F03BC1822F90E0FC013A97A1
:10365000EF36F10508F02CC1EC5CFF4F0C94ED2F18
:1036600085E396E069E471E0A7C085E396E065E54F
:1036700071E00E94FB2C85E78983DE011296E3EB63
:10368000F3E08BE101900D928150E1F7CE010196BC
:103690006CE10E94EF0F0E947E0C83E08093980300
:1036A00068EC70E080E090E00E94F429809198033B
:1036B000843009F0FDC08FE70E94900A0E94A40A9E
:1036C0008983853509F0F4C085E396E06FED74E0F9
:1036D0000E94852B85E396E061EC74E00E94852BC7
:1036E00085E396E063EA74E0ACC085E396E06DE6BE
:1036F00071E00E94FB2C89E68983CE01019661E08E
:103700000E94EF0F0E947E0C83E08093980368EC88
:1037100070E080E090E00E94F4298091980384306A
:1037200009F0C6C08FE70E94900A0E94A40A89830C
:103730008E010E5F1F4F2DE1E22EF12CEC0EFD1ECF
:103740000E94A40AD8018D938D01AE15BF05C1F763
:10375000A3EBB3E0FE0132968BE101900D92815014
:10376000E1F78981893409F0A3C085E396E065E833
:1037700074E00E94852B85E396E067E674E00E9482
:10378000852B85E396E069E474E05BC085E396E011
:1037900067E871E00E94FB2C8EEF8093230488C0C1
:1037A00020522750922F905380912004891738F48B
:1037B00085E396E066E971E00E94FB2C79C0909366
:1037C00023046FC084E18093230485E396E062E1E3
:1037D00074E037C085E18093230485E396E06BEDC8
:1037E00073E02FC086E18093230485E396E064EACA
:1037F00073E027C087E18093230485E396E06AE5C0
:1038000073E01FC088E18093230485E396E069E4B8
:1038100073E017C089E18093230485E396E065E3B4
:1038200073E00FC08AE18093230485E396E060E2B1
:1038300073E007C08BE18093230485E396E068EF93
:1038400072E00E94852B34C085E396E06EED72E055
:103850000E94852B8091C10391E01DC085E396E015
:1038600068EC72E00E94852B8091C10392E013C046
:1038700085E396E063EB72E00E94852B8091C103A3
:1038800094E009C085E396E068E972E00E94852B28
:103890008091C10398E089278093C1038FEF8093C3
:1038A00023040E946D1A04C085E396E00E947A2EDC
:1038B00085E396E00E94402E892BB1F762C1822FEA
:1038C0000E94CC16882309F45CC180918904882366
:1038D00021F48FEF809323044CC184E294E060E0F4
:1038E00070E040E050E00E94A2069B01AC016091B4
:1038F0002304862F992787FD9095A92FB92FFC01C6
:103900003197EB31F10508F024C1ED55FF4F0C94D0
:10391000ED2FE62FFF27E7FDF0958091200490E042
:103920008E179F070CF415C1DA01C9010197A1098F
:10393000B1098097A105B10548F098E2F92E00E0A1
:1039400010E06F010894C108D10825C0ED54FC4F68
:10395000822F81508083E5C0612F70E0660F771F52
:1039600061507C4FFB01808190E08C159D0591F4A6
:103970008F2D90E0A0E0B0E082179307A407B50771
:1039800041F4F601ED54FC4FDB0111968C918183DB
:1039900001E0F3941F5F80911F041817E8F2BFC085
:1039A0002F3F31054105510511F008F0D2C0209399
:1039B000CB03B7C02F3F31054105510511F008F089
:1039C000C8C02093CC03ADC02F3F31054105510540
:1039D00011F008F0BEC02093CD03A3C08091240451
:1039E0008062803719F585E294E060E070E040E0A5
:1039F00050E00E94A2069B01AC01DC01CB010197C3
:103A0000A109B1090897A105B10508F0B5C0CA011F
:103A1000B90124ED30E340E050E00E94472F9B01C4
:103A2000AC012A5E3C4A4A46554E24C0863611F502
:103A300085E294E060E070E040E050E00E94A20681
:103A40009B01AC01DC01CB010197A109B1090797EA
:103A5000A105B10508F090C0CA01B90128EA31E614
:103A600040E050E00E94472F9B01AC01245E3C43A4
:103A70004E46544E211531054105510561F0DA01DC
:103A8000C90180509447AB48B24381509A45A24641
:103A9000B24008F05EC02093C3033093C403409348
:103AA000C5035093C6033DC02F3F31054105510565
:103AB00011F008F04EC02093C70333C0DA01C901EA
:103AC0000197A109B1098F3F9105A105B10508F042
:103AD00040C02093C80325C0DA01C901845C994025
:103AE000A040B0408D549D41A040B04030F4309390
:103AF000CA032093C90301E001C000E0211531058C
:103B00004105510511F48FEF07C0213431054105FE
:103B1000510528F4822F81508093C20302C00023F4
:103B2000C1F080918A048823D1F48091D7039091C9
:103B3000D803A091D903B091DA030196A11DB11D5C
:103B40008093D7039093D803A093D903B093DA035B
:103B500006C085E396E068EA71E00E94FB2C0E94B3
:103B6000C2168FEF8093230485E396E06AE00E94FB
:103B7000992B0E946D1A05C021E030E040E050E032
:103B80007ECF6C96E8E00C94DC2F85E396E06CE445
:103B900072E00E94852B85E396E064E372E00E9468
:103BA000852B85E396E00E94402E892B31F085E33A
:103BB00096E00E947A2E0E94181B0E94EE1482301A
:103BC00019F0833069F405C085E396E066E172E0A0
:103BD00004C085E396E06FEF71E00E94852B0895A5
:103BE0008FEF8093230410928A040E946D1A0CC0F8
:103BF00085E396E00E94402E892B31F085E396E024
:103C00000E947A2E0E94181B809123048E3F81F718
:103C1000089580912304992787FD9095A92FB92FA6
:103C2000FC013196EB30F10508F074C0E254FF4F0F
:103C30000C94ED2F85E396E064E678E00E94852BF6
:103C400083E793E00E943C1A85E396E06CE478E019
:103C50000E94852B85E396E067E278E00E94852B41
:103C600085E396E06DEF77E00E94852B85E396E093
:103C70006CED77E00E94852B85E396E06FEA77E0B4
:103C80000E94852B85E396E069E877E00E94852B0A
:103C900085E396E065E677E00E94852B85E396E074
:103CA0006EE377E00E94852B85E396E00E946F2B00
:103CB0000E9415192FC085E396E061E277E028C0E5
:103CC00085E396E06CEF76E023C085E396E067EE4F
:103CD00076E01EC085E396E068EC76E019C085E3E7
:103CE00096E064E876E014C085E396E06FE676E05F
:103CF0000FC085E396E06AE576E00E94852B85E3B8
:103D000096E064E176E004C085E396E06EEF75E04E
:103D10000E94852B6AE070E080E090E00E94F42928
:103D200004C085E396E00E947A2E85E396E00E9427
:103D3000402E892BB1F70895A2E2B0E0E2EAFEE15D
:103D40000C94B62F8E010F5F1F4F80E1D8011D929A
:103D50008A95E9F785E396E066EC71E00E94FB2C1A
:103D60000E949A1520E034E74BE852E32F8F38A3E6
:103D700049A35AA380E09EECADEEB4E38B8F9C8FF9
:103D8000AD8FBE8F24EF31E040E050E02F8B388FB5
:103D9000498F5A8F60E5C62E63ECD62EE12CF12CAC
:103DA000412C54E7552E5BE8652E52E3752E88248E
:103DB0009924540133241E8A1D8A198A1A8A1B8A5F
:103DC0001C8AFFC085E396E00E947A2E8434B9F005
:103DD000853430F48332B9F18C3209F0CCC044C060
:103DE000833509F0C8C02F8D38A149A15AA1C90156
:103DF000DA012C013D01882499245401E2C085E3B5
:103E000096E064E40E94672B85E396E040E054E787
:103E10006BE872E32AE030E00E949B2C85E396E099
:103E20006CE20E94672B85E396E040E05EEC6DEE6D
:103E300074E32AE030E00E949B2C85E396E06CE27C
:103E40000E94992BBEC019821A821B821C821D827D
:103E50001E821F82188619861A861B861C861D865E
:103E60001E861F86188A3AC0339434E0331609F050
:103E7000A8C069817A818B819C8128EE33E040E083
:103E800050E00E94472F6F8F78A389A39AA36D817A
:103E90007E818F8198850E94472F6B8F7C8F8D8FBD
:103EA0009E8F89859A85AB85BC858F8B988FA98FCE
:103EB000BA8F6D857E858F8598890E94472F6B010B
:103EC0007C0190E2C9169EE4D90690E0E90690E0F4
:103ED000F90630F48CE162E30E94BA0A332471C01F
:103EE000A0E3CA16A5E7DA06A0E0EA06A0E0FA0613
:103EF00018F48CE162E2F0CFB0E4CB16BCE9DB064B
:103F0000B0E0EB06B0E0FB0618F48CE166E2E4CF2B
:103F1000E0E5CE16E3ECDE06E0E0EE06E0E0FE06CD
:103F200018F48CE162E1D8CFF0E6CF16FAEEDF06A6
:103F3000F0E0EF06F0E0FF0618F48CE165E1CCCF8D
:103F400020E7C21621E1D20621E0E20620E0F206D7
:103F500018F48CE161E0C0CF30EAC31636E8D3062E
:103F600031E0E30630E0F30618F48CE163E0B4CF0F
:103F70008CE165E0B1CF40ED242E280E49E04215DA
:103F800000F1032D10E0000F111F000F111F81E041
:103F900090E08C0F9D1F080F191FD8016D917D9126
:103FA0008D919C912AE030E040E050E00E94472F44
:103FB000620D711D811D911DF801608371838283E3
:103FC000938385E396E00E94402E892B09F0FACE78
:103FD00081149104A104B10489F4C301B2010E94C7
:103FE000300B61E070E080E090E00E94F429FFEF88
:103FF000FE8B1D8A198A1A8A1B8A1C8A2F89388D82
:10400000498D5A8D82169306A406B506E0F40E94E7
:10401000DB0A29893A894B895C89280F311D411DAA
:10402000511D298B3A8B4B8B5C8B3D89381708F4DB
:104030008D8B4E89841708F48E8B0894811C911CFB
:10404000A11CB11C56C0C301B20128EE33E040E010
:1040500050E00E94792F85E396E0BA01A9012AE099
:1040600030E00E942D2C85E396E06CE20E94672BE5
:1040700085E396E06D894AE050E00E94752C85E367
:1040800096E06CE20E94672B69897A898B899C890A
:10409000A50194010E94792F85E396E0BA01A90158
:1040A0002AE030E00E942D2C85E396E06CE20E942D
:1040B000672B85E396E06E894AE050E00E94752CFC
:1040C00085E396E06CE20E94992B4C0C5D1C6E1C03
:1040D0007F1C8B8D9C8DAD8DBE8D84159505A605A1
:1040E000B70520F44F8C58A069A07AA088249924A1
:1040F00054012F8D38A149A15AA1285E3340404078
:10410000504009F05ECFA296E2E10C94D22FA0E0DD
:10411000B0E0EDE8F0E20C94C12F0E94CE296115C9
:10412000710581059105C9F30E9499061092D70384
:104130001092D8031092D9031092DA03DD24E09094
:10414000D703F090D8030091D9031091DA03102F10
:104150000F2DFE2CEE240E9494062FEF30E040E05D
:1041600050E00E949B2FE60EF71E081F191FE092D9
:10417000D703F092D8030093D9031093DA03D394B2
:1041800044E0D416E1F6CDEDD3E000E010E070E1BC
:10419000E72E77E2F72E4EC00F5F19F40E944D080C
:1041A0004DC00E94940622E330E040E050E00E94BF
:1041B0009B2F6F5FEDEDF3E090E004C081918617D7
:1041C00059F39F5F9117D0F38091DC0390E08E9DAF
:1041D00090018F9D300D9E9D300D1124862F90E013
:1041E000AC01249FC001259F900D349F900D112498
:1041F000AA2797FDA095BA2F2091D3033091D4031D
:104200004091D5035091D603820F931FA41FB51F71
:1042100020919B0330919C0340919D0350919E03FC
:10422000281739074A075B0708F4B6CF69931F5F61
:10423000183121F08881882309F0AECFCDB7DEB7E1
:10424000E7E00C94DD2F80E060E00E94F115882308
:1042500031F081E060E00E94F115882341F40E9472
:1042600092080E944D080E9487200E949716089588
:10427000AAE5B0E0EEE3F1E20C94C22F8B017A01E3
:104280008B3009F426C18C3040F5853009F484C0A8
:10429000863080F4823009F459C0833020F48130B4
:1042A00009F050C242C0833009F461C0843009F083
:1042B00049C265C0883009F49DC0893038F4863021
:1042C00009F486C0873009F03DC28CC0893009F4FA
:1042D00099C08A3009F036C2C9C0893609F482C152
:1042E0008A3680F4863609F42DC1873620F4853667
:1042F00009F028C20EC1873609F43DC1883609F09D
:1043000021C241C18C3609F4C4C18D3638F48A36D5
:1043100009F473C18B3609F015C2AFC18D3609F4AB
:10432000ECC1873C09F00EC200C281E069E270E096
:104330000E94A7110EEC13E0F80181918F010E94F9
:104340009011F3E0073F1F07B9F704C282E06BE169
:1043500070E00E94A71103EB13E0F80181918F0137
:104360000E949011F3E00E3C1F07B9F7F3C183E000
:1043700061E070E00E94A7110E94EE14E9C184E0A0
:1043800061E070E00E94A71181E00E9490110E94FC
:1043900089110E949C1EE0C160911F0470E0660FAD
:1043A000771F85E00E94A71100E010E008C0F80127
:1043B000E150FC4F80810E9490110F5F1F4F809150
:1043C0001F0490E0880F991F0817190780F3C2C1D6
:1043D00086E062E070E00E94A71183E793E00E940C
:1043E0009E11B8C187E061E070E00E94A711809142
:1043F0002004AEC188E061E070E00E94A7118091C6
:104400009903A6C186E68983CE01019661E00E94E8
:10441000EF0F0E947E0C83E08093980368EC70E0BD
:1044200080E090E00E94F429809198038430E1F4C8
:104430008FE70E94900A0E94A40A8983863471F44F
:1044400089E060E270E00E94A71110E00E94A40AD7
:104450000E9490111F5F1032C9F77CC189E061E0B2
:1044600070E00E94A711C7C089E06DC18AE069E1D0
:1044700070E00E94A71181E080939A0380919F05CC
:10448000882351F080919F039091A003A091A103F4
:10449000B091A203806809C080919F039091A0030E
:1044A000A091A103B091A2038F7780939F03909373
:1044B000A003A093A103B093A2030AE913E0F801BB
:1044C00081918F010E949011F3E0033B1F07B9F720
:1044D00041C18BE061E270E00E94A7118091BE04AF
:1044E0008F3F39F08091BE048F5F8093BE0481506E
:1044F00002C08091BE040E94901110E0812F0E94A2
:10450000950D0E94190A0E949E111F5F1031B1F78C
:1045100021C185E661E070E00E94A7110932110512
:1045200009F015C120E030E0F901E253FC4FD7015A
:10453000A20FB31F8C9180832F5F3F4F293231052B
:1045400099F759C086E661E070E00E94A7110B312F
:10455000110509F0FCC020E030E0F901ED54FC4FFA
:10456000D701A20FB31F8C9180832F5F3F4F2B3158
:10457000310599F740C087E661E070E00E94A7111D
:104580000E94971638C088E661E070E00E94A7118B
:1045900085E78A83DE011396E3EBF3E08BE101907C
:1045A0000D928150E1F7CE0102966CE10E94EF0F6F
:1045B0000E947E0C83E08093980360E273E080E0C9
:1045C00090E00E94F42980919803843009F0BFC0E4
:1045D0008FE70E94900A0E94A40A8A83853509F019
:1045E000B6C009C089E661E070E00E94A7110E9490
:1045F0004D080E94920881E0ABC08AE661E070E05D
:104600000E94A71189E68E8FCE014E9661E00E942E
:10461000EF0F0E947E0C83E08093980360E273E0CA
:1046200080E090E00E94F42980919803843009F0A2
:104630008EC08FE70E94900A0E94A40A8E8F8E017E
:10464000015E1F4FFAE3EF2EF12CEC0EFD1E0E94CF
:10465000A40AF80181938F01EE15FF05C1F7A3EBC2
:10466000B3E0FE017F968BE101900D928150E1F75E
:104670008E8D893409F06BC0BECF8BE661E070E0AF
:104680000E94A711F70180810E94B2160E94232187
:10469000B2CF8CE661E070E00E94A71100321105F4
:1046A00071F487E68AAFDE01DB96F70180E20190C4
:1046B0000D928150E1F7CE01CA9661E205C087E410
:1046C0008AAFCE01CA9661E00E94EF0F0E947E0C75
:1046D00083E0809398036CE474E080E090E00E94B3
:1046E000F42980919803843091F58FE70E94900A15
:1046F0000E94A40A873459F57ECF8DE661E070E010
:104700000E94A7110931110511F520E030E0F901EF
:10471000E656FC4FD701A20FB31F8C9180832F5F09
:104720003F4F2931310599F766CF87EC61E070E0A2
:104730000E94A71181E00E9490110E94891110929D
:10474000FD030AC08AEC61E070E00E94A71180E0DE
:104750000E9490110E948911C65ADF4FE6E00C9426
:10476000DE2FA0E0B0E0E7EBF3E20C94BE2F54E0C4
:10477000A52E46E0B42E35E0C32E03E315E024E673
:10478000D22E92E0E92E83E0F82EA1C085E396E0D8
:104790000E947A2E982F80939E0580919D058330EC
:1047A00021F1843028F4813099F08230B8F409C0C6
:1047B000853009F448C0853020F1863009F087C083
:1047C0005FC0953B09F083C081E080939D057FC069
:1047D000923609F07AC0E0929D0579C090939C05CD
:1047E00090939B05F0929D0572C09093990510924D
:1047F0009A0580919B05892780939B05A0929D0532
:1048000066C0D92FC0E02091990530919A052C2BD4
:104810003D2B30939A052093990580919B0589271C
:1048200080939B05C0929D052536310508F44FC045
:104830008CEC61E070E00E94A71181E00E94901171
:104840000E94891142C02091970530919805F90185
:10485000ED5CFA4F908380919B05892780939B059F
:104860002F5F3F4F309398052093970580919905CE
:1048700090919A052817390750F1B0929D0527C0ED
:1048800080919B05891759F460919705709198055F
:1048900080919C0543E355E00E9438210DC08BECCC
:1048A00062E070E00E94A71180919C050E94901127
:1048B0008091FE030E949011F8018D2D11928A952E
:1048C000E9F7109298051092970510929D0585E3DF
:1048D00096E00E94402E892B09F058CFCDB7DEB765
:1048E000EAE00C94DA2F81E08093FD0308C085E3B1
:1048F00096E00E94402E892B11F00E94B1238091F6
:10490000FD038823A1F708951F93109123041F3FEF
:1049100009F0F1C0893409F467C08A3428F5883376
:1049200009F479C0893368F4803309F486C081338F
:1049300008F06FC08B3109F44DC0813209F0D5C049
:104940003DC0813409F49AC0823438F4893309F4C3
:1049500072C0803409F0C9C031C0823409F4A1C0EA
:10496000863409F0C2C052C0823609F49AC0833638
:1049700090F4883579F1893538F4823509F43FC0EF
:10498000833509F0B2C01FC08A3509F4A9C0813649
:1049900009F0ABC073C0823791F1833730F48636AB
:1049A000A9F1893609F0A1C01FC0883799F08A376C
:1049B00009F496C0833709F098C005C085E396E0F6
:1049C00069E471E019C00E94971685E396E063EDF3
:1049D00071E006C00E94232185E396E06DEE71E050
:1049E0000E94FB2C8EEF7FC00E944D080E9492080F
:1049F00085E396E06CE072E00E94FB2C76C00E949A
:104A0000872085E396E065E272E0F6CF0E943517D5
:104A10006CC0805368C085E396E06CEE71E00E9444
:104A2000852B9091F603892F885F8871977E892B5B
:104A30008093F60320C089E056C085E396E069EDD7
:104A400071E00E94852B80919F039091A003A0911B
:104A5000A103B091A20320E130E040E050E08227C2
:104A60009327A427B52780939F039093A003A09337
:104A7000A103B093A2031093230437C085E396E00B
:104A800063EC71E00E94852B80919F039091A003BD
:104A9000A091A103B091A20320E430E040E050E0F7
:104AA00012C085E396E062EB71E00E94852B809155
:104AB0009F039091A003A091A103B091A20320E2D3
:104AC00030E040E050E082279327A427B527809369
:104AD0009F039093A003A093A103B093A20302C0ED
:104AE0000E94C51D8FEF80932304809123048E3F85
:104AF00009F4DDC0D4C00E94CC16882309F4D7C0C5
:104B000080918904882321F48FEF80932304C7C008
:104B100084E294E060E070E040E050E00E94A20691
:104B20009B01AC0180912304992787FD9095A92FC3
:104B3000B92FFC013197E930F10508F08CC0E7533B
:104B4000FF4F0C94ED2FDA01C90181509447AB4817
:104B5000B2438F5F9945A246B24008F07CC02093D3
:104B6000D3033093D4034093D5035093D6039AC014
:104B70002093D7033093D8034093D9035093DA039B
:104B800081E080938A048EC02830310541055105AB
:104B900008F061C02093DB0385C0DA01C9010197E9
:104BA000A109B1090A97A105B10508F054C02093E5
:104BB000DC0378C084E294E06DE371E00E94BE07FC
:104BC00010E00EC0183130F4E12FF0E0E253FC4F5A
:104BD00087871F5F80E090E06DE371E00E94BE0771
:104BE000009759F00E94A007009761F706C0E12FD7
:104BF000F0E0E253FC4F17861F5F1831C0F352C03C
:104C0000253031054105510530F52093F5034AC0A3
:104C1000DA01C9010197A109B1090697A105B105FA
:104C2000D0F48091F603887F822B8093F6033AC0FC
:104C3000DA01C9010197A109B1098050924CA14044
:104C4000B04048F42093CF033093D0034093D10376
:104C50005093D20327C085E396E068EA71E00E9492
:104C6000FB2C13C08091D7039091D803A091D90356
:104C7000B091DA030196A11DB11D8093D7039093E3
:104C8000D803A093D903B093DA030E94C2168FEF22
:104C90008093230485E396E06AE00E94992B0E94AA
:104CA000091E05C080918A048823E1F2EECF1F918E
:104CB00008958FEF8093230410928A040E94091EA6
:104CC0000CC085E396E00E94402E892B31F085E3ED
:104CD00096E00E947A2E0E948424809123048E3FC5
:104CE00081F76AE070E080E090E00E94F42904C05F
:104CF00085E396E00E947A2E85E396E00E94402E9E
:104D0000892BB1F70895AAE2B0E0E9E8F6E20C9445
:104D1000BB2F0E94C0297B018C0181E00E949F0B68
:104D200004C085E396E00E947A2E85E396E00E9417
:104D3000402E892BB1F72C98DD24D394E2E67E2E09
:104D400072E0872E912C8C0E9D1E5E010894A11C92
:104D5000B11C63E0C62E0E94C02920E030E06E192D
:104D60007F09800B910B693C71058105910510F05D
:104D700021E030E08D2D90E028233923232B99F179
:104D80000E94C0297B018C012B9A80ED97E00E9444
:104D9000DB117982D401EEECF3E089E201900D920F
:104DA0008150E1F7C5016AE20E94EF0F2B9880E085
:104DB00090E00E94DB11C09298030E947E0C62E397
:104DC00070E080E090E00E94F429809198038430A4
:104DD00051F4C09298038FE70E94900A0E94A40A9F
:104DE000823409F4DD248AE00E94F22A892B49F5F5
:104DF000DD24D39426C02C9A2B9A85E396E00E945A
:104E00007A2E8D30910569F08E3091051CF40A9749
:104E1000B1F407C08332910569F08234910579F4C9
:104E20000CC085E396E064EA71E00E94852B0E9445
:104E3000592605C00E949C1E02C00E9473242C9813
:104E40002B9885E396E00E94402E892B09F483CFAE
:104E5000D2CF8F929F92AF92BF92CF92DF92EF927A
:104E6000FF920F931F938AE00E94F22A892B09F088
:104E700083C068EC70E080E090E00E94F42980E05C
:104E800090E00E94DB110E94C0295B016C01F0ECF4
:104E9000EF2EF2E1FF2E012D112DE60EF71E081F59
:104EA000191F06C08AE00E94F22A892B09F062C00D
:104EB0000E94C0296E157F058007910798F38AE04C
:104EC0000E94F22A892B09F055C080ED97E00E94DC
:104ED000DB110E94C0297B018C01992493948824C2
:104EE00088E496E2A0E0B0E0A80EB91ECA1EDB1E60
:104EF00029C0AE14BF04C006D10638F480ED97E097
:104F00000E94DB11882483941DC00E94C0296E1961
:104F10007F09800B910B693C71058105910590F02B
:104F20000E94C0297B018C0180E0992009F481E076
:104F3000982E882319F480E090E002C080ED97E07D
:104F40000E94DB118AE00E94F22A892B91F280E014
:104F500090E00E94DB11882049F0809199038F5FD7
:104F600083700E94B2160E94232106C00E948720EF
:104F70000E9497160E9483261F910F91FF90EF9039
:104F8000DF90CF90BF90AF909F908F90089581E079
:104F90006DEF77E042E050E00E94FB280895EF9229
:104FA000FF920F931F9380E00E9419080E94C61180
:104FB0008CE061E00E94532A8BE061E00E94532A5A
:104FC0008AE060E00E94532A83E160E00E94532A55
:104FD00083E161E00E94BF2A82E161E00E94532ADE
:104FE00082E160E00E94BF2A0E94C61485E396E039
:104FF00040E052EC61E070E00E94B92D0E94A516DD
:105000000E9423210E94740D8FEF8093BE040E94A2
:10501000C72778940E94C0297B018C018091BE042F
:105020008F3F09F0DEC00E94C0296E197F09800BF6
:10503000910B605D77408040904008F0D2C0EECF89
:1050400085E396E00E947A2E85E396E00E94402E4A
:10505000892BB1F785E396E062E472E00E94F82CB8
:1050600083E793E00E943C1A85E396E069E572E0ED
:105070000E94F82C85E396E060E070E04AE050E0A2
:105080000E94E42C62E370E080E090E00E94F4294A
:1050900085E396E00E94402E04970CF185E396E0AC
:1050A0000E947A2E82349105D1F485E396E00E9425
:1050B0007A2E8E34910599F485E396E00E947A2E3B
:1050C0008434910561F485E396E00E947A2E8197FD
:1050D00031F480E090E00E94DB110E948326409131
:1050E000CF035091D0036091D1037091D203DB01C3
:1050F000CA010197A109B1090497A105B10568F496
:105100004093BF04433029F040E052EC61E070E08E
:1051100004C040EA56E861E070E085E396E00E9452
:10512000B92D0E9429272C9880E090E00E94DB1185
:105130000E94740D1092A30480919F0383FF11C0FD
:105140008091E303882351F08091EA03882331F0B2
:105150008091F103882311F087E001C085E08093FE
:10516000A30480E00E949F0B8091A2040E94C50AC4
:105170000E947E0C10922705109228051092290596
:1051800010E015C062E370E080E090E00E94F42936
:1051900080ED97E00E94DB1162E370E080E090E038
:1051A0000E94F42980E090E00E94DB111F5F809153
:1051B0009903811738F78091F60390E084FF09C0C6
:1051C00020E088719070489709F421E0822F0E94B6
:1051D000CF148FE00E9419081F910F91FF90EF905C
:1051E000089580ED97E00E94DB118AE061E00E9463
:1051F000BF2A2C9A29CF823000F5E82FF0E0EE0F7D
:10520000FF1FE056FA4F71836083882319F08130C5
:10521000A1F408C0809169008C7F842B8093690081
:10522000E89A089580916900440F551F440F551F57
:10523000837F842B80936900E99A08951F920F92CF
:105240000FB60F9211242F933F934F935F936F9359
:105250007F938F939F93AF93BF93EF93FF9380912F
:10526000A0059091A105892B29F0E091A005F0916E
:10527000A1050995FF91EF91BF91AF919F918F91FA
:105280007F916F915F914F913F912F910F900FBE42
:105290000F901F9018951F920F920FB60F92112426
:1052A0002F933F934F935F936F937F938F939F932E
:1052B000AF93BF93EF93FF938091A2059091A305C5
:1052C000892B29F0E091A205F091A3050995FF91A2
:1052D000EF91BF91AF919F918F917F916F915F916E
:1052E0004F913F912F910F900FBE0F901F901895E7
:1052F0001F920F920FB60F9211242F933F938F930B
:105300009F93AF93BF938091A8059091A905A09119
:10531000AA05B091AB053091AC050196A11DB11D58
:10532000232F2D5F2D3720F02D570196A11DB11D84
:105330002093AC058093A8059093A905A093AA0596
:10534000B093AB058091A4059091A505A091A60509
:10535000B091A7050196A11DB11D8093A40590935E
:10536000A505A093A605B093A705BF91AF919F9106
:105370008F913F912F910F900FBE0F901F90189516
:105380008FB7F8942091A8053091A9054091AA05FE
:105390005091AB058FBFB901CA0108959FB7F8942A
:1053A0002091A4053091A5054091A6055091A7052F
:1053B00086B5A89B06C08F3F21F02F5F3F4F4F4F10
:1053C0005F4F9FBF542F432F322F2227280F311DAD
:1053D000411D511D82E0220F331F441F551F8A9526
:1053E000D1F7B901CA010895EF92FF920F931F936D
:1053F000CF93DF937B018C010E94CE29EB010EC07D
:105400000E94CE296C1B7D0B685E7340C8F3089424
:10541000E108F10801091109C851DC4FE114F10458
:105420000105110569F7CDB7DEB7E6E00C94DE2F74
:10543000789484B5826084BD84B5816084BD85B56F
:10544000826085BD85B5816085BDEEE6F0E0808136
:1054500081608083E1E8F0E0108280818260808357
:10546000808181608083E0E8F0E0808181608083DA
:10547000E1EBF0E0808184608083E0EBF0E080810C
:1054800081608083EAE7F0E08081846080838081AE
:105490008260808380818160808380818068808356
:1054A0001092C1000895CF93DF93482F50E0CA01B6
:1054B0008D5F934FFC0134914151544FFA01849117
:1054C000882369F190E0880F991FFC01EF52F44F97
:1054D000A591B491FC01E552F44FC591D491662396
:1054E00051F42FB7F8948C91932F909589238C9336
:1054F000888189230BC0623061F42FB7F8948C91B6
:10550000932F909589238C938881832B88832FBF39
:1055100006C09FB7F8948C91832B8C939FBFDF912B
:10552000CF910895833071F0843028F48130A1F058
:10553000823021F514C08630B1F08730D1F084304C
:10554000E9F404C0809180008F7703C080918000CF
:105550008F7D80938000089584B58F7702C084B5D5
:105560008F7D84BD08958091B0008F778093B000C7
:1055700008958091B0008F7D8093B0000895FF92D0
:105580000F931F93F62E482F50E0CA01895E934F68
:10559000FC012491CA018D5F934FFC01149141518C
:1055A000544FFA0104910023C9F0222319F0822FED
:1055B0000E94922AE02FF0E0EE0FFF1FE552F44F19
:1055C000A591B4919FB7F894FF2021F48C91109588
:1055D000812302C08C91812B8C939FBF1F910F91CF
:1055E000FF9008950F931F93482F50E0CA01895EE2
:1055F000934FFC012491CA018D5F934FFC010491EC
:105600004151544FFA011491112319F420E030E074
:1056100015C0222319F0822F0E94922A812F90E038
:10562000880F991F8B51944FFC01A591B4918C91D7
:1056300020E030E0802311F021E030E0C9011F912B
:105640000F910895A0E0B0E0E8E2FBE20C94C02FD7
:105650007C016B018A01C0E0D0E00FC0D6016D91E2
:105660006D01D701ED91FC910190F081E02DC70112
:105670000995C80FD91F015010400115110571F788
:10568000CE01CDB7DEB7E8E00C94DC2FEF92FF92AD
:105690000F931F93CF93DF937C018B01C0E0D0E089
:1056A000F8010F5F1F4F6491662359F0D701ED9108
:1056B000FC910190F081E02DC7010995C80FD91F19
:1056C000EFCFCE01CDB7DEB7E6E00C94DE2FDC01E4
:1056D000ED91FC910190F081E02D09950895EF92F4
:1056E000FF920F931F938C016DE00E94672B7C014A
:1056F000C8016AE00E94672B9C012E0D3F1DC90165
:105700001F910F91FF90EF900895EF92FF920F93EA
:105710001F937C010E94462B8C01C7010E946F2BB6
:105720009C01200F311FC9011F910F91FF90EF9035
:105730000895EF92FF920F931F937C010E94672BB5
:105740008C01C7010E946F2B9C01200F311FC901E2
:105750001F910F91FF90EF900895CF93DF93EC018D
:105760006115710519F420E030E00FC0DB010D90E8
:105770000020E9F71197A61BB70BE881F981028099
:10578000F381E02DAD0109959C01C901DF91CF9115
:1057900008954F925F927F928F929F92AF92BF92A5
:1057A000CF92DF92EF92FF920F931F93DF93CF93ED
:1057B000CDB7DEB7A1970FB6F894DEBF0FBECDBF51
:1057C0002C01742ECB01223008F42AE019A231E218
:1057D000C32ED12CCC0EDD1E822E9924AA24BB24EC
:1057E000672D752FA50194010E94792F79018A01F7
:1057F000C801B701A50194010E94472F472D461B00
:105800000894C108D1084A3010F4405D01C0495CD9
:10581000F6014083E114F1040105110521F07E2C0D
:105820005F2DC801DDCFC201B6010E94AD2BA1964C
:105830000FB6F894DEBF0FBECDBFCF91DF911F91A1
:105840000F91FF90EF90DF90CF90BF90AF909F901F
:105850008F907F905F904F900895DC012115310566
:1058600041F4ED91FC910190F081E02D642F0995B8
:1058700008950E94C92B0895EF92FF920F931F93F2
:105880007C010E942D2C8C01C7010E946F2B9C0172
:10589000200F311FC9011F910F91FF90EF900895C4
:1058A000EF92FF920F931F939A017B0100E010E0AB
:1058B000B801A7010E942D2C1F910F91FF90EF902E
:1058C0000895EF92FF920F931F937C010E94502C3A
:1058D0008C01C7010E946F2B9C01200F311FC90151
:1058E0001F910F91FF90EF900895EF92FF920F9309
:1058F0001F939A01E62EFF2400E010E0B801A701F3
:105900000E942D2C1F910F91FF90EF900895EF9220
:10591000FF920F931F937C010E94752C8C01C7018D
:105920000E946F2B9C01200F311FC9011F910F9105
:10593000FF90EF900895A0E0B0E0E1EAFCE20C9463
:10594000C02FEC016A017B012115310541F4E8818A
:10595000F9810190F081E02D642F09951BC02A3058
:105960003105B1F477FF13C06DE20E94672B8C0103
:1059700044275527BA014C195D096E097F09CE01EC
:105980002AE00E94C92B9C01200F311F04C02AE08D
:105990000E94C92B9C01C901CDB7DEB7E8E00C9489
:1059A000DC2FEF92FF920F931F937B019A01002748
:1059B000F7FC0095102FB801A7010E949B2C1F91A6
:1059C0000F91FF90EF900895EF92FF920F931F9326
:1059D0007C010E94D12C8C01C7010E946F2B9C017D
:1059E000200F311FC9011F910F91FF90EF90089573
:1059F0000E94AD2B0895EF92FF920F931F937C01AD
:105A00000E94F82C8C01C7010E946F2B9C01200F73
:105A1000311FC9011F910F91FF90EF9008950895D4
:105A20001F920F920FB60F9211242F933F934F9313
:105A30008F939F93EF93FF938091C00082FD1DC0D1
:105A40004091C6002091ED053091EE052F5F3F4F4C
:105A50002F7330708091EF059091F005281739076A
:105A600071F0E091ED05F091EE05E355FA4F4083BA
:105A70003093EE052093ED0502C08091C600FF91A2
:105A8000EF919F918F914F913F912F910F900FBE6A
:105A90000F901F9018951F920F920FB60F9211241E
:105AA0002F933F938F939F93EF93FF932091310612
:105AB00030913206809133069091340628173907C9
:105AC00031F48091C1008F7D8093C10014C0E091BA
:105AD0003306F0913406EF50FA4F2081809133065F
:105AE0009091340601968F73907090933406809352
:105AF00033062093C600FF91EF919F918F913F91C4
:105B00002F910F900FBE0F901F901895A0E0B0E05E
:105B1000ECE8FDE20C94BC2FFC011382128288EEAB
:105B200093E0A0E0B0E084839583A683B7838AE8FE
:105B300093E0918380837587648757874687318B8D
:105B4000208B138B028BF58AE48AD78AC68AB18EA2
:105B5000A08E938E828E8F85848F8889858F898988
:105B6000868F8A89878F8B8980A32096ECE00C949E
:105B7000D82FAF92BF92DF92EF92FF920F931F93B5
:105B8000CF93DF93EC017A018B01DD24403081EE6D
:105B9000580780E0680780E0780711F0DD24D3948F
:105BA00091E0A92EB12CEC89FD89DD2069F0C501B9
:105BB00008A002C0880F991F0A94E2F7808360E072
:105BC00079E08DE390E005C0108260E874E88EE132
:105BD00090E0A80197010E94792F21503040404069
:105BE0005040569547953795279580E120303807E6
:105BF00020F0DD2011F0DD24D6CFE889F98930834B
:105C0000EA89FB89208319A2EE89FF89408121E07E
:105C100030E0C9010C8C02C0880F991F0A94E2F78A
:105C2000482B4083EE89FF894081C9010D8C02C059
:105C3000880F991F0A94E2F7482B4083EE89FF8969
:105C40004081C9010E8C02C0880F991F0A94E2F7A7
:105C5000482B4083EE89FF8980810F8C02C0220F80
:105C6000331F0A94E2F7209528232083DF91CF91F8
:105C70001F910F91FF90EF90DF90BF90AF9008952C
:105C8000DC011C96ED91FC911D97E05CFF4F21918A
:105C9000319180819181281B390B2F733070C9019C
:105CA000089585E396E00E94402E892B11F00E9412
:105CB0000F2D0895DC011C96ED91FC911D97E05C81
:105CC000FF4F20813181E054F040DF01AE5BBF4FD8
:105CD0008D919C9111972817390719F42FEF3FEFF9
:105CE00007C08D919C91E80FF91F8081282F30E02B
:105CF000C9010895DC011C96ED91FC911D97E05CB3
:105D0000FF4F20813181E054F040DF01AE5BBF4F97
:105D10008D919C9111972817390719F42FEF3FEFB8
:105D200010C08D919C911197E80FF91F20818D91E2
:105D30009C91119701968F73907011969C938E93FE
:105D400030E0C9010895DC0191968C9191978823E8
:105D500039F05496ED91FC915597808186FFF9CFEB
:105D600091961C920895CF93DF93EC01EE85FF8509
:105D7000E05CFF4F20813181E054F0402F5F3F4FC6
:105D80002F733070DF01AE5BBF4F8D919C911197E7
:105D900028173907D1F3E05CFF4F80819181E054EF
:105DA000F040E80FF91F6083EE85FF85E05CFF4F50
:105DB00031832083EE89FF89208181E090E00F8C80
:105DC00002C0880F991F0A94E2F7282B208381E0F4
:105DD00089A3EC89FD8980818064808381E090E0E3
:105DE000DF91CF9108958F929F92AF92BF92CF9201
:105DF000DF92EF92FF920F931F9300D000D00F928B
:105E0000EDB7FEB7319684E0ADB7BEB711968C936F
:105E100083E0818387E0828385E0838381E08483DC
:105E200085E396E06DEA75E041EF55E025EC30E062
:105E300004EC10E0B0ECEB2EF12CA1ECCA2ED12C2E
:105E4000F2ECAF2EB12CE6EC8E2E912C0E94862D1A
:105E50000F900F900F900F900F901F910F91FF9048
:105E6000EF90DF90CF90BF90AF909F908F9008956C
:105E7000CF93DF930E94182A0E94CF27C1E5DEE26C
:105E80000E94E5112097E1F30E94512EF9CF629F05
:105E9000D001739FF001829FE00DF11D649FE00D22
:105EA000F11D929FF00D839FF00D749FF00D659F83
:105EB000F00D9927729FB00DE11DF91F639FB00D82
:105EC000E11DF91FBD01CF011124089597FB092E93
:105ED00007260AD077FD04D086D006D000201AF419
:105EE000709561957F4F0895F6F7909581959F4F36
:105EF0000895A1E21A2EAA1BBB1BFD010DC0AA1F0B
:105F0000BB1FEE1FFF1FA217B307E407F50720F022
:105F1000A21BB30BE40BF50B661F771F881F991F9D
:105F20001A9469F760957095809590959B01AC01E6
:105F3000BD01CF01089597FB092E05260ED057FD10
:105F400004D0D7DF0AD0001C38F450954095309526
:105F500021953F4F4F4F5F4F0895F6F790958095ED
:105F6000709561957F4F8F4F9F4F08952F923F926D
:105F70004F925F926F927F928F929F92AF92BF9259
:105F8000CF92DF92EF92FF920F931F93CF93DF9305
:105F9000CDB7DEB7CA1BDB0B0FB6F894DEBF0FBE62
:105FA000CDBF09942A88398848885F846E847D84AF
:105FB0008C849B84AA84B984C884DF80EE80FD80B1
:105FC0000C811B81AA81B981CE0FD11D0FB6F89427
:105FD000DEBF0FBECDBFED010895EE0FFF1F059090
:105FE000F491E02D0994AA1BBB1B51E107C0AA1F25
:105FF000BB1FA617B70710F0A61BB70B881F991F6A
:106000005A95A9F780959095BC01CD0108959111FD
:1060100006C0803219F089508550D0F7089599272D
:0860200088270895F894FFCFD2
:106028004E6F005965730054582074696D656F751B
:106038007421006D6F64756C65206C6F636B6564AB
:106048003F00486F70206368616E6E656C200020A9
:1060580040200053004E2F4100386368002C002C6C
:10606800205B005D20280029004E4F5420454E41FA
:10607800424C45440053656E64696E6720736574CD
:1060880074696E677320746F2052580A00526573E2
:10609800657474696E672073657474696E677320BC
:1060A8006F6E2052580A0041626F727465642065F1
:1060B800646974730A00696E76616C69642073653B
:1060C8006C656374696F6E000D0A496E76616C6960
:1060D8006420696E707574202D2064697363617221
:1060E8006465642107007363616E6E6572206D6F6D
:1060F80064650053657474696E67732073617665AF
:106108006420746F20454550524F4D0A0052657601
:1061180065727465642073657474696E677320664C
:10612800726F6D20454550524F4D0A004C6F6164A7
:10613800656420666163746F727920646566617551
:106148006C74730A004B657920616E642063686122
:106158006E6E656C732072616E646F6D697A6564CA
:106168000A004F70656E4C52536E67205458207366
:1061780074617274696E672000206F6E2048572022
:106188000050504D0052535349005344410053436B
:106198004C00525844005458440041494E004C4267
:1061A8004545500053504B54524D005342555300EF
:1061B80053554D44004C4C494E440000342B340098
:1061C8003800382B340031320031322B340031366C
:1061D8000001000000C01200001A400AA1204EA5CC
:1061E800001B1E27522C23308025000005400AA1E1
:1061F800204EA50020244EA52C2330004B0000067D
:10620800400AD0009D49007B289D492C233000E19D
:10621800000005400A4501D7DC03B81E0EBF002365
:106228002E48E801008A400A6001555502AD1E203B
:10623800000023C88025000005400AA1204EA500C3
:1062480020244EA52C233000020002000200020088
:106258000200020002000200020002000200020026
:1062680002000200020002FF610265026A026E0279
:10627800720276027A027E0284028B0290029502F2
:106288009B029B029B029B0235019C02A002A20278
:10629800A602A902AE02350100070B0C1011150069
:1062A800160A1322312900000000B32E222B402E9B
:0662B8007A2E5A2EA32EDF
:00000001FF
